:100000000C94EB040C9413050C9413050C94130539
:100010000C9413050C9413050C9413050C94130500
:100020000C9413050C9413050C94B01F0C941F2012
:100030000C9413050C9413050C9413050C941305E0
:100040000C9413050C9413050C9413050C941305D0
:100050000C9413050C9413050C9413050C94512265
:100060000C9413050C9413050C9413050C941305B0
:100070000C9413050C9413050C9413050C941305A0
:100080000C9413050C9413050C9413050C94130590
:100090000C9413050C9413050C9413050C94130580
:1000A0000C9413050C9413050C941305AA55AA552A
:1000B000AA55AA55080800000054007C00380038F2
:1000C000007C00540000000E005800700030003822
:1000D0000078005800100000004C005E00570257E6
:1000E0000077002200000006006C00380018001C99
:1000F000007E044E000C0004001E007C0038003816
:10010000007C001E00040010009800CB007F007FE0
:1001100000CB00980010009200D6007C007E007E8C
:10012000007C00D60092000C0078003E047F047F23
:10013000003E0078000C0007008C00FC003F003FF0
:1001400000FC008C0018000F005C00F800BC007F71
:1001500004DF008E000C0033009A00FF047F047F50
:1001600000FF009A0033FFFFFFFFFFFFFFFFFF8349
:10017000C1E1E1C183FFFF83F9FDFDF983FFFFFFCB
:10018000FFAA55FFFFFFF7EFF7EFF7EFF7EFFFFFDE
:10019000FFFAF5EBF7EFFFFFFFBF5FAFD7EFF7EB2E
:1001A000F5FAFDFFFFFFF7EFD7AF5FFFFFFFFFFFA0
:1001B000FFAA55EFF7EFF7EFF7AF57EFF7EFF7EFCE
:1001C000F7AA55FFFFFFF7EFF7EAF5EFF7EFF7EFC5
:1001D000F7AA55EFF7EF00000000003E5B4F5B3ED3
:1001E0003E6B4F6B3E1C3E7C3E1C183C7E3C181CFC
:1001F000577D571C1C5E7F5E1C00183C1800FFE7F3
:10020000C3E7FF0018241800FFE7DBE7FF30483A98
:10021000060E2629792926407F050507407F0525FA
:100220003F5A3CE73C5A7F3E1C1C08081C1C3E7F82
:1002300014227F22145F5F005F5F06097F017F0049
:100240006689956A606060606094A2FFA294080469
:100250007E040810207E201008082A1C08081C2A8A
:1002600008081E101010100C1E0C1E0C30383E38E2
:1002700030060E3E0E06000000000000005F000089
:100280000007000700147F147F14242A7F2A1223FA
:100290001308646236495620500008070300001C0A
:1002A0002241000041221C002A1C7F1C2A08083E13
:1002B0000808008070300008080808080000606026
:1002C0000020100804023E5149453E00427F400094
:1002D00072494949462141494D331814127F10276C
:1002E000454545393C4A49493141211109073649BB
:1002F000494936464949291E00001400000040348F
:100300000000000814224114141414140041221493
:100310000802015909063E415D594E7C1211127CBA
:100320007F494949363E414141227F4141413E7F1B
:10033000494949417F090909013E414151737F08FB
:1003400008087F00417F41002040413F017F0814A1
:1003500022417F404040407F021C027F7F04081002
:100360007F3E4141413E7F090909063E4151215EE0
:100370007F09192946264949493203017F01033F74
:100380004040403F1F2040201F3F4038403F631403
:1003900008146303047804036159494D43007F4105
:1003A00041410204081020004141417F0402010242
:1003B0000440404040400003070800205454784067
:1003C0007F284444383844444428384444287F38FB
:1003D0005454541800087E090218A4A49C787F087D
:1003E00004047800447D40002040403D007F1028F8
:1003F000440000417F40007C047804787C080404B9
:10040000783844444438FC1824241818242418FC50
:100410007C08040408485454542404043F44243CF5
:100420004040207C1C2040201C3C4030403C442864
:100430001028444C9090907C4464544C44000836FE
:10044000410000007700000041360800020102046C
:10045000023C2623263C1EA1A161123A4040207A8C
:1004600038545455592155557941215454784121D6
:100470005554784020545579400C1E52721239550B
:100480005555593954545459395554545800004508
:100490007C410002457D420001457C40F029242931
:1004A000F0F0282528F07C545545002054547C5405
:1004B0007C0A097F49324949493232484848323238
:1004C0004A4848303A4141217A3A42402078009DDA
:1004D000A0A07D39444444393D4040403D3C24FF88
:1004E0002424487E4943662B2FFC2F2BFF0929F635
:1004F00020C0887E090320545479410000447D4186
:100500003048484A32384040227A007A0A0A727DDE
:100510000D19317D2629292F2826292929263048F9
:100520004D4020380808080808080808382F10C867
:10053000ACBA2F102834FA00007B000008142A14EB
:100540002222142A14089500220095AA005500AA18
:10055000AA55AA55AA000000FF00101010FF0014B1
:100560001414FF001010FF00FF1010F010F014140E
:1005700014FC001414F700FF0000FF00FF1414F433
:1005800004FC141417101F10101F101F1414141F34
:1005900000101010F0000000001F101010101F10AD
:1005A000101010F010000000FF10101010101010AC
:1005B0001010FF10000000FF140000FF00FF0000FB
:1005C0001F10170000FC04F414141710171414F46F
:1005D00004F40000FF00F714141414141414F700AA
:1005E000F7141414171410101F101F141414F414FB
:1005F0001010F010F000001F101F0000001F14006A
:100600000000FC140000F010F01010FF10FF141494
:1006100014FF141010101F00000000F010FFFFFF67
:10062000FFFFF0F0F0F0F0FFFFFF0000000000FF20
:10063000FF0F0F0F0F0F38444438447C2A2A3E1412
:100640007E02020606027E027E026355494163383D
:1006500044443C04407E201E2006027E020299A5EE
:10066000E7A5991C2A492A1C4C7201724C304A4D4C
:100670004D303048784830BC625A463D3E49494981
:10068000007E0101017E2A2A2A2A2A44445F44442A
:1006900040514A444040444A51400000FF0103E0B9
:1006A00080FF000008086B6B083612362436060FF0
:1006B000090F06000018180000001010003040FF5D
:1006C0000101001F01011E00191D1712003C3C3CD6
:1006D0003C0000000000F0F89C8E8783878E9CF819
:1006E000F00000FEFF0303030303070EFCF8000005
:1006F000FEFF0303030303070EFCF80000FFFF00E7
:10070000000000000000FFFF0000FEFF83838383E2
:1007100083C7EE7C380000F8FC0E07030303070EC6
:10072000FCF800003F7FE0C08080C0E07F3FFFFF1B
:1007300001010101010101FFFF0000FFFF0C0C0C92
:100740000C1C3E77E3C100007FFFC0C0C0C0C0E00A
:10075000703F1F00001F3F70E0C0C0C0E0703F1F2F
:1007600000007FFFC1C1C1C1C1E3773E1C00001F73
:100770003F70E0C0C0C0E0703F1F000000000001FB
:10078000FFFF01000000D5F08D14A1C881CFD9F181
:10079000AF20005265616C6C793F20413D79204269
:1007A0003D6E006E6577207265636F72642100672D
:1007B000616D65206F7665722061742000636865E5
:1007C00061742100191C1C1C1C191313070707074F
:1007D0001313191010FFFF3F3F8793B9E5E5B99355
:1007E000873F3FFFFFFFFFFF8E96B096BFBF96B0DB
:1007F000968EFFFFFFFFFF3FBF878381999981831B
:1008000087BF3FFFFFFFFFFF8EA680A08080A080F4
:10081000A68EFFFFFFFFFFFFE3C91D73E7E7731D10
:10082000C9E3FFFFFFFFFFFB91A4B495BFBF95B4E1
:10083000A491FBFFFFFFFFFFE3C91933070733193B
:10084000C9E3FFFFFFFFFFFB95A484A48E8EA48461
:10085000A495FBFFFFF763B75F5B4140415B5F58C7
:10086000414041585F5B4140415B5FAF47EF80557E
:10087000803E7F416F6F717F3E0003017F01030067
:100880007F41633E807F800303020100010001007D
:100890000100010001000100010001000102030349
:1008A000080B00020202000009040000010202001D
:1008B000000524001001052401010104240206059D
:1008C000240600010705810310004009040100020D
:1008D0000A000000070502024000000705830240ED
:1008E00000000403090412010002EF020140412349
:1008F000368000010102030141726475696E6F2048
:100900004C4C43004142413133303600FFC399E53E
:10091000E599C3FFFFC199F3F399C1FFFFFFFBF90D
:10092000FBEF87FFFFFBF9FBFF97A7FFFFBB93C719
:10093000C793BBFFFFFFFF81C3E7FFFFFFC399B56D
:10094000AD99C3FFFFE783818183E7FFFFE78B8DCD
:100950008D8BE7FFFFE783B1B183E7FFFF998181CB
:10096000818199FFFF99858D8D8599FFFF99A1B1AF
:10097000B1A199FFFF8F838181838FFFFF8F838DCB
:100980008D838FFFFF8FB3B1B1B38FFFFF9381834F
:10099000838193FFFF938D8B8B8D93FFFF93A1B387
:1009A000B3A193FFFFF181838381F1FFFFF18D8B71
:1009B0008B8DF1FFFFF181B3B381F1FFFFEB8181FB
:1009C0008181EBFFFFEB858D8D85EBFFFFEB91B117
:1009D000B191EBFFCE2211241FBECFEFDAE0DEBFD4
:1009E000CDBF11E0A0E0B1E0E4EAFEE502C0059071
:1009F0000D92A839B107D9F729E0A8E9B1E001C003
:100A00001D92A630B207E1F714E0CBEED4E004C0AB
:100A10002197FE010E94722CCA3ED107C9F70E949D
:100A2000D0230C94502F0C940000AF92BF92CF9221
:100A3000DF92EF92FF920F931F93CF93DF93CDB787
:100A4000DEB72F970FB6F894DEBF0FBECDBFA982D9
:100A5000BA82CB82DC82ED82FE820F8318872987DF
:100A60003A874B875C876D877E878F8780913F06AB
:100A7000823078F49FE0989FD0011124FE013196D6
:100A8000AF5DB94F01900D929A95E1F78F5F80931A
:100A90003F062F960FB6F894DEBF0FBECDBFDF9195
:100AA000CF911F910F91FF90EF90DF90CF90BF906B
:100AB000AF900895480F592F511D1416150694F53F
:100AC000803891057CF597FF02C090E080E04138C6
:100AD000510514F040E850E0481BFB01E770FF2788
:100AE00021E030E001C0220FEA95EAF7209577FF78
:100AF00002C0695F7F4FFB0133E0F595E7953A95BA
:100B0000E1F7F695FE2FEE27F795E795E80FF91F29
:100B1000E553FE4F415030F08191DF011197822360
:100B20008C93F8CF08956F927F928F929F92AF929D
:100B3000BF92CF92DF92EF92FF920F931F93CF93CA
:100B4000DF937C01FA011491319654913196C12FB3
:100B5000D0E0222309F1CC24C394D12C852F8770B7
:100B600011F4D12CC12CA52FA695A695A695AC0D58
:100B7000BD2DB11DAC9FC001AD9F900DBC9F900DD0
:100B80001124033011F4880F991F289FD001299F49
:100B9000B00D1124EA0FFB1FD701AC0FBD1F1A16B1
:100BA0001B060CF0FAC080E8E816F1040CF0F5C062
:100BB000CB01850F911D181619060CF0EEC060349C
:100BC00071050CF0EAC0309709F4E7C0362F377092
:100BD000CB0177FD079623E0959587952A95E1F758
:100BE000282F77FF04C0332311F02FEF280F66273B
:100BF00077276E197F09F7FC02C070E060E090E88B
:100C00009E19A038B1050CF4912F961B41E02E3FA0
:100C100009F040E0BB24B394852F877009F4B12C10
:100C2000569556955695B50EAB2DB0E0A20FB11D59
:100C300027FDBA9519971CF058E0B52EB21AB41AD0
:100C4000240F50E82503D0011124AE0DBF1DA60FBF
:100C5000B71FE42EF12CEC9EA001ED9E500DFC9EE2
:100C6000500D1124460F571FC32E032E000CDD0814
:100C7000033009F445C04E0F5F1F6FEF70E0032E85
:100C800002C0660F771F0A94E2F760957095972E61
:100C90008B2C820E281509F480C08D0105531E4F40
:100CA000F12CE12CE91630F5FA01EE0DFF1DE4916F
:100CB000F0E03F010C2C02C0660C771C0A94E2F7AE
:100CC00027FD05C0F8018081862386298083332390
:100CD00059F027304CF45801F0E8AF0EB11CF50183
:100CE0008081892187298083FFEFEF1AFF0A0F5F38
:100CF0001F4FD8CF2F5F4C0F5D1FA058BF4FCACFDB
:100D0000E92EF12C440F551FE40FF51FA553BE4FDC
:100D100060E870E06E197F09CE19DF098E01000FBF
:100D2000111F41E050E07A01032E01C0EE0C0A943D
:100D3000EAF7592F4B2D892E932ECF93DF93ED0198
:100D4000EF96EF962296A590C590992059F0AE9C0B
:100D50005001CE9C600127302CF4F880D094FD2007
:100D6000FB28F99222233AF0FC90C094FC20FA2848
:100D7000FD920C94BC0611965A9529F74A9551F0AC
:100D8000582D23951124E00FF11DA60FB11DC60F9C
:100D9000D11DD9CFDF91CF911124DF91CF911F9138
:100DA0000F91FF90EF90DF90CF90BF90AF909F900A
:100DB0008F907F906F90089590E0EBECF1E09111AF
:100DC0009FEF8FEF91939193919391938150D0F7EF
:100DD0000895EBECF1E0A0E0B8E000800EBC8111DA
:100DE000012C1197A0FDFDCF0192B9F70DB4089524
:100DF000FC018091CA01882311F13FB7F89482E089
:100E00008093E9002091F200822F90E018161906D5
:100E100014F481E090E0882339F0289844E6409368
:100E2000C9014091F1004083222339F02091F20062
:100E3000211103C02BE62093E8003FBF08958FEFF8
:100E40009FEF08952FB7F89483E08093E900909185
:100E5000E800892F807295FF04C09091F20080E431
:100E6000891B2FBF08958091C10181110DC082E0BF
:100E70008093BD0184E08093BE011092C001109266
:100E8000BF0181E08093C1018DEB91E00895CF9384
:100E9000DF931F92CDB7DEB76983DC01ED91FC9142
:100EA0000280F381E02D41E050E0BE016F5F7F4F93
:100EB00009950F90DF91CF91089583E08093E90029
:100EC0008091F200882319F08AE38093E800089566
:100ED0000E94220790E00895CF93DF931F92CDB731
:100EE000DEB7FC018485958597FD08C02FEF3FEFA5
:100EF000358724870F90DF91CF910895CE01019619
:100F00000E94F806019719F4898190E0F3CF8FEFE2
:100F10009FEFF0CF0F931F93CF93DF931F92CDB727
:100F2000DEB78C01FC018485958597FF0BC0CE014F
:100F300001960E94F806019771F4898190E0F8010A
:100F400095878487F801848595850F90DF91CF91EF
:100F50001F910F9108958FEF9FEFF1CFFC018485D2
:100F6000958597FD0BC09FB7F89482E08093E900C8
:100F70008091F2009FBF90E0019608959FB7F8948A
:100F800082E08093E9008091F2009FBF90E0089595
:100F90004091B7015091B8012091B5013091B6014F
:100FA00042175307B4F49091E8009570E1F39091E3
:100FB000E80092FD19C08093F1008091B7019091F3
:100FC000B80101968F739927892B19F48EEF8093BE
:100FD000E8008091B7019091B80101969093B80113
:100FE0008093B70181E0089580E00895DF92EF9249
:100FF000FF920F931F93CF93DF93D82E8A01EB01BB
:101000007B01E40EF51ECE15DF0559F0D7FE12C0A8
:10101000FE0184910E94C80721968111F4CF0FEF41
:101020001FEFC801DF91CF911F910F91FF90EF90BB
:10103000DF9008958881EECF0F931F93CF93DF93B6
:101040001F92CDB7DEB782E0898342E450E060EAC8
:1010500078E080E80E94F6070E943307DC011296D0
:101060000D911C910115110589F0D801ED91FC91AC
:101070000280F381E02DBE016F5F7F4FC8010995AB
:1010800097FD04C0F80100851185ECCF89810F9090
:10109000DF91CF911F910F910895615030F0209111
:1010A000F100FC0120830196F8CF289884E6809314
:1010B000C9010895FC010E94F108319728F0685198
:1010C0007C4F8F4F9F4FF9CFAB01FC010E94F1087D
:1010D000641775078E079F07C8F308958F929F9234
:1010E000AF92BF92CF92DF92EF92FF920F931F9336
:1010F000CF93DF936C017B018A0180910E018823DD
:1011000009F45AC08091CA01882309F455C080911E
:10111000BC0180FF05C08091E00082608093E00008
:10112000E801B12C8AEFA82E93E0892E2AE3922EB3
:10113000209711F4BB20C9F10E942207811108C039
:10114000AA94AA20C9F181E090E00E945A08F0CF49
:101150008C171D0611F00CF08C2F9FB7F89480921D
:10116000E9002091E80025FD02C09FBFE1CF282FB4
:1011700030E0C21BD30BF701815020F04191409326
:10118000F100FACFE20EF31EBB2021F09092E800AE
:10119000B12CEBCF8091E80085FDE7CF9092E8007D
:1011A000BB24B394209709F3F3CF5D9884E6809332
:1011B000BB01101611063CF081E090E0F60193832C
:1011C000828310E000E0C801DF91CF911F910F9161
:1011D000FF90EF90DF90CF90BF90AF909F908F9057
:1011E0000895A1EBB1E02FB7F8947D918D919C917A
:1011F00066B52FBFA89B05C06F3F18F47F5F8F4F68
:101200009F4F22E0660F771F881F991F2A95D1F7FD
:101210000895AF92BF92CF92DF92EF92FF920F9319
:101220001F93CF93DF936C017B018B01040F151F7C
:10123000EB015E01AE18BF08C017D10759F06991E4
:10124000D601ED91FC910190F081E02DC601099548
:10125000892B79F7C501DF91CF911F910F91FF90F5
:10126000EF90DF90CF90BF90AF90089590E00C94F6
:101270005A088FB18095807F669B88601C9B846034
:1012800008951092A2013E98579808953E9A579A51
:1012900081E08093A2010895CF93C82F0E9439095D
:1012A000982F9C2381E09C1380E0CF91089580E0EB
:1012B0000C94E9062F923F924F925F926F927F9229
:1012C0008F929F92AF92BF92CF92DF92EF92FF9256
:1012D0000F931F93CF93DF9300D000D0CDB7DEB72D
:1012E0006E2C30E0F901E80FF91F1E161F060CF0F6
:1012F00095C0803891050CF091C0402E512CF20120
:10130000E60FF71F1E161F060CF088C0603471052B
:101310000CF084C0E62FE7707E2EF7E04F0E511CD4
:10132000E3E055944794EA95E1F7F3E07595679506
:10133000FA95E1F7A62E660FBB08B5017695762FD4
:10134000662777956795680F791F65537E4FDA0199
:1013500010E000E07801EA0CFB1C48E0E416F10420
:101360000CF05CC0EFEFEE16FE060CF44DC09C8353
:101370008B8350E040E04B01F0E88F0E911CCB8056
:10138000DC80D7FC31C0FD01E40FF51FE491F0E0F3
:101390006F01072C02C0CC0CDD1C0A94E2F7DA8244
:1013A000C982EFEFEE16FE0609F456C06B01C40EBB
:1013B000D51EF6013080F1E06F1247C0E9813E2A68
:1013C000F6013082772081F0F7E0EF16F10461F04A
:1013D0006401C40ED51EF6013080F1E0EA816F127F
:1013E00038C03E2AF60130824F5F5F4FEB81FC81AF
:1013F0003196FC83EB834217530734F4EB81FC8175
:10140000E038F10509F0BBCF0F5F1F4F60587F4FE9
:10141000A20FB31F4016510609F09CCF0F900F90FA
:101420000F900F90DF91CF911F910F91FF90EF9050
:10143000DF90CF90BF90AF909F908F907F906F90F4
:101440005F904F903F902F900895298020943220F4
:10145000B7CFE0953E22C6CF7110BACFC5CF803846
:101460009105B8F460347105A0F490E121E061FDCC
:1014700024E060FD220F62FD2295687F969FD001D7
:101480001124A80FA553BE4F0C90022A40FF02263C
:101490000C9208952F923F924F925F926F927F929B
:1014A0008F929F92AF92BF92CF92DF92EF92FF9274
:1014B0000F931F93CF93DF9300D000D0CDB7DEB74B
:1014C0007C018B01242F30E03C832B8381E090E072
:1014D0005C01A21AB30A1901319421943108220C3B
:1014E000331CB901600F711F40E0C7010E942F0A31
:1014F000B8018B819C81681B790B40E0C7010E9479
:101500002F0A40E0B8018B819C818E0D9F1D0E94A7
:101510002F0A40E0B801C7012B813C81821B930B4D
:101520000E942F0AD12CC12C81E090E09A838983FC
:101530002B813C81C216D3060CF05DC0B7FC09C0FC
:10154000215031093C832B8332E0230E311CA20C45
:10155000B31C8FEFC81AD80A29813A812E5F3F4FFA
:101560003A832983A20EB31E37016C0C7D1C40E028
:101570008B809C80800E911EB401C3010E942F0AB3
:1015800027014C185D0840E0B401C2010E942F0AF7
:1015900040E048018B819C81881A990AB401C301FB
:1015A0000E942F0A40E0B401C2010E942F0A4601A6
:1015B000800E911E40E0B4016B807C806E0C7F1C1D
:1015C000C3010E942F0A40E0B40127012B813C8116
:1015D000421A530AC2010E942F0A48018C189D0822
:1015E00040E0B401C3010E942F0A40E0B401C201EF
:1015F0000E942F0A9DCF0F900F900F900F90DF91B8
:10160000CF911F910F91FF90EF90DF90CF90BF90FF
:10161000AF909F908F907F906F905F904F903F9092
:101620002F9008952F923F924F925F926F927F92E8
:101630008F929F92AF92BF92CF92DF92EF92FF92E2
:101640000F931F93CF93DF93EC018B017A01690114
:10165000C61AD70AD7FE03C0D194C194D108470156
:101660008C1A9D0A97FE03C09194819491088C1462
:101670009D0454F49E2D8F2D7901292F382F9C2FF6
:101680008D2FE801092F182FEC16FD0654F4902F2A
:10169000812F8901292F382F9C2F8D2FE701E92ECB
:1016A000F82E17012C1A3D0A2901401A510A57FE3B
:1016B00003C0519441945108310137FE03C08FEFAC
:1016C000681A780A759467948FEF021713070CF461
:1016D00081E0A82E880FBB08EC16FD06A4F040E0C0
:1016E000BE01C8018C149D0414F0B801CE010E9403
:1016F0002F0A6418750877FE04C00A0D1B1D620CC2
:10170000731C2196E9CFDF91CF911F910F91FF902C
:10171000EF90DF90CF90BF90AF909F908F907F9091
:101720006F905F904F903F902F9008955F926F92CF
:101730007F928F929F92AF92BF92CF92DF92EF9261
:10174000FF920F931F93CF93DF936D3089F0C0907A
:10175000A601D090A7016A30E9F41092A501109279
:10176000A40188E0C80ED11CD092A701C092A601A6
:1017700081E090E0DF91CF911F910F91FF90EF906A
:10178000DF90CF90BF90AF909F908F907F906F90A1
:101790005F9008956090A301509002010091A40110
:1017A0001091A501E5E06E9FE0011124CA52DE4FC1
:1017B0005801F12CF5E0E12CFF1629F0CE0101963D
:1017C000FE01E490EC01460188E0782EE0FC18C0B0
:1017D000462D651016C0E6947A94FFEF8F1A9F0A83
:1017E0007110F4CFF3948FEFA81AB80AE6E0FE1256
:1017F000E1CF0A5F1F4F1093A5010093A401B8CF5A
:10180000452DB401C5010E942F0AE5CF0F931F9308
:10181000CF93DF938C01D0E0C0E0F801EC0FFD1F07
:101820006491662341F08CE196E00E94960B892B2F
:1018300011F02196F2CFCE01DF91CF911F910F9140
:101840000895DF92EF92FF920F931F93CF93DF9350
:101850007C01D22E8B01040F111DEB0177FF02C01A
:10186000D0E0C0E0C8010134110514F080E490E03C
:10187000C817D9073CF44D2DBE01C7010E942F0A9D
:101880002196F0CFDF91CF911F910F91FF90EF90B4
:10189000DF900895EF92FF920F931F93CF93DF9302
:1018A0007C018B01C42FD22F6034710510F40E948B
:1018B0005A05B8016D0F711D6150710960347105D1
:1018C00020F44C2FC7010E945A0520E04D2FB8018B
:1018D000C7010E94210CC7018C0F911D20E04D2FE4
:1018E000B8010197DF91CF911F910F91FF90EF9079
:1018F0000C94210CCF92DF92EF92FF920F931F93E3
:10190000CF93DF936B01122FEC017C01E40EF11CED
:10191000CE15DF0544F4202F412FB601CE010E94E1
:10192000210C2196F5CFDF91CF911F910F91FF9060
:10193000EF90DF90CF9008950F931F93CF93DF9395
:1019400000D000D01F92CDB7DEB749835A836B8396
:101950007C838D83F8014081518180E042335105C1
:10196000A8F485E0849FD001859FB00D1124A20FBB
:10197000B31FFE01319601900D928A95E1F7F801AF
:101980008081918101969183808381E00F900F90F7
:101990000F900F900F90DF91CF911F910F910895AD
:1019A0002F923F924F925F926F927F928F929F926F
:1019B000AF92BF92CF92DF92EF92FF920F931F935D
:1019C000CF93DF93CDB7DEB728970FB6F894DEBF7D
:1019D0000FBECDBF6E834F83322EE8862601282EA0
:1019E00082E3821510F482E3282EC02ED12CEE243F
:1019F000FF24EC18FD08712C612C362D621408F0C0
:101A000042C0862D68850E943E2C20E0911107C0BF
:101A1000EC18FD08232DE3E0E31508F423E0F201C0
:101A2000668D832F0E943E2CE92F4E814B3008F0AB
:101A30004AE06F816B3008F06AE0641B770B6F5FE0
:101A40007F4FC3010E945E2C480F7E2DFD82EC82E9
:101A5000F4E04F9FD0011124A652B74F11965C912C
:101A60005F7380E4289F90011124522B4F70EC1873
:101A7000FD08840195016E2F8D810E949C0CEFEF73
:101A80006E1A7E0ABACF28960FB6F894DEBF0FBE44
:101A9000CDBFDF91CF911F910F91FF90EF90DF901D
:101AA000CF90BF90AF909F908F907F906F905F90FE
:101AB0004F903F902F900895CF93DF9300D000D0A8
:101AC00000D01F92CDB7DEB7877097E0899FF001F5
:101AD0001124E95DFE4F87E0DE01119601900D9221
:101AE0008A95E1F729813A814B815C816D817E8104
:101AF0008F8190E027960FB6F894DEBF0FBECDBF62
:101B0000DF91CF9108954F925F926F927F928F9263
:101B10009F92AF92BF92CF92DF92EF92FF920F937C
:101B20001F93CF93DF9300D000D000D01F92CDB78A
:101B3000DEB78C01F62E2CE0261708F4A6C1FC01B6
:101B400010821382E090D1084090D2088E2C912C04
:101B5000F0E14F9E300111246401C60CD71C5601E0
:101B6000AA0CBB1CC5018C0D9D1DFC01E05EF94F4C
:101B700056A42EE0521229C0815B994FFC0180814E
:101B80000E945C0D29833A834B835C836D837E8343
:101B90008F832F2D30E0F5E0FF1510F148E1F49E22
:101BA000C00111248C5B964FF80192838183511000
:101BB0005FC087E0829FF001839FF00D1124E95DF3
:101BC000FE4F8481F801838378C087E0E7E2F1E08B
:101BD000DE01119601900D928A95E1F768E0D9CF68
:101BE000C90173E0880F991F7A95E1F78452974FE6
:101BF000F80192838183F7E0FF1508F44AC1511080
:101C000037C0EE20A9F1442099F1EA94EE2DF0E0DE
:101C10006E0E7F1ED301AA0FBB1FA60DB71DA05EBF
:101C2000B94F9E968C91811123C04A9440E1449E05
:101C3000C0011124880E991ED401AA0FBB1FA80D44
:101C4000B91DA05EB94F9E964C91411111C08E0FE7
:101C50009F1FFC01EE0FFF1FE80FF91FE05EF94F19
:101C600081E096A5911101C080E0F8018083A1CFA9
:101C700081E0FBCFF501EC0DFD1DE15BF94F20810B
:101C800030E0F8E080E890E0FF1611F080E490E0AA
:101C900028233923232B21F081E0F80180830DC014
:101CA000FEE05F12F9CF862F90E0880F991F63E066
:101CB00070E00E945E2CF8016383F9E0FF12F6C029
:101CC000F501EC0DFD1DE15BF94F808187708650B9
:101CD000823008F0EBC0E7C087E6F801848385E72F
:101CE000858381E6868382E7878384E68087118601
:101CF0000CC083E6F801848381E685838EE68683C3
:101D000087839FE6908781871286C80127960FB642
:101D1000F894DEBF0FBECDBFDF91CF911F910F9121
:101D2000FF90EF90DF90CF90BF90AF909F908F90FB
:101D30007F906F905F904F90089589E6F8018483BB
:101D400083E6858385E686831782DFCF85E6F80103
:101D500084839CE69583868383E6878384E78087F4
:101D600082E7D1CF83E7F80184838EE6858389E615
:101D7000868380E7878385E6F2CF8DE6F80184834A
:101D800081E6858387E6868389E6878383E6AECF0F
:101D900087E7F801848381E6858384E7868385E687
:101DA000878382E7A3CF86E6F801848389E685836B
:101DB00082E7868385E687831086A7CFF501EC0D41
:101DC000FD1DE05EF94F86A58E30A9F481E090E01C
:101DD000F8E0FF1202C090E080E08C0F9D1FFC0134
:101DE00086819BE2F8019483823049F138F488239C
:101DF000D1F08130F1F0F801148287CF833019F1EE
:101E00008430C9F783E7848380E7858384E686830B
:101E100080E2878381E6808795E7918792E79287C2
:101E20008387148672CF84E685838DE6868387E672
:101E3000C2CF83E7858380E7868384E6BCCF82E7D1
:101E400085838EE6F3CF83E7848388E685838FE6F8
:101E5000868383E687838BE649CF83E7F801848313
:101E600085E685838CE68683A6CF87E6F8018483A2
:101E70008FE6858381E267CF81E7F801848385E778
:101E8000858389E6868384E796CF82E0F8018083A4
:101E9000B3CFF9E0FF1508F0EDCE2AE0F21216C03C
:101EA000FEE05F1619F081E0F8018083F8012381DC
:101EB0008091CC089091CD082817190639F030F0A0
:101EC00080914C06813011F081E08083EFEFEF0DBF
:101ED000EC3008F001CFF0E0E059F04F0C94722C98
:101EE000790E9D0EA60EB20EBD0EC80ED30EDE0EDE
:101EF000DE0E2D0F350F3C0F82E08093CB0580E482
:101F00008093900087E597E09093990080939800E4
:101F100008958F929F92AF92BF92CF92DF92EF92ED
:101F20000F931F93CF93DF93FB016A01EB0183E0D3
:101F3000D695C7958A95E1F7CB01880F991F880F31
:101F4000991F65E070E00E944A2C42E0460FCF01E5
:101F500063E070E00E944A2CCF01049648015901C9
:101F600054E0E52E0AE02C2F880F0E94D00CDF9160
:101F7000CF911F910F91EF90DF90CF90BF90AF90D6
:101F80009F908F9008958F929F92AF92BF92CF9221
:101F9000DF92EF920F931F93FB016A0159019B019E
:101FA00083E0369527958A95E1F7CB01880F991F35
:101FB000880F991F65E070E00E944A2C462FCF01E0
:101FC00063E070E00E944A2C8E2F880F480154E095
:101FD000E52E07E08D5F0E94D00C1F910F91EF90CE
:101FE000DF90CF90BF90AF909F908F9008952F92E9
:101FF0003F924F925F926F927F928F929F92AF9299
:10200000BF92CF92DF92EF92FF920F931F93CF93E5
:10201000DF93CDB7DEB729970FB6F894DEBF0FBEBA
:10202000CDBF6B012A0149013801CB0101968232F3
:10203000910510F081E290E08887C60167E070E0CA
:102040000E944A2C6987C60163E070E00E944A2C16
:102050006E836B3010F02AE02E83C601880F991F23
:1020600063E070E00E944A2C6B3008F06AE0862F33
:10207000EE818E1B990B1C01FFEF2F1A3F0AF12CEA
:10208000E12C86EFA82EBB24BA94EF828885E8164F
:1020900008F046C09BEAE99E812D11248695982F71
:1020A000990F890F20E08E1106C02985ECE1CE162C
:1020B000D10408F023E0C701B1010E945E2C4E81DB
:1020C000480F7A2DBD82AC8284E0489FF001112434
:1020D000E652F74F51815F7390E4299F90011124DC
:1020E000522B5A834F7049838301940160E0EAE0E8
:1020F000AE1AB1088D810E949C0CF201868D82304F
:1021000058F0FF81F0FD08C0940149815A8161E0D7
:102110007C818D810E949C0C2FEFE21AF20AB5CFD0
:1021200029960FB6F894DEBF0FBECDBFDF91CF91D9
:102130001F910F91FF90EF90DF90CF90BF90AF90E5
:102140009F908F907F906F905F904F903F902F90D7
:1021500008958F929F92AF92BF92CF92DF92EF92AB
:102160000F931F93FB016A01CB0165E070E00E94B1
:102170004A2C4E2FEF30F10520F4E930F10508F03C
:1021800048E0CF0196958795969587954801590126
:1021900075E0E72E0AE0262F682F81E08E0F0E945F
:1021A000D00C1F910F91EF90DF90CF90BF90AF9028
:1021B0009F908F900895CF93DF9300D000D000D0F0
:1021C0001F92CDB7DEB7FC0120812E3039F481811A
:1021D0000E945C0D265081E0223008F080E02796B6
:1021E0000FB6F894DEBF0FBECDBFDF91CF9108953B
:1021F0000F931F93CF93DF9300D000D000D01F9296
:10220000CDB7DEB7062FFC011081812F0E945C0D37
:102210008F83701303C081E017FD06C08F81801388
:102220000EC016FB882780F927960FB6F894DEBFFC
:102230000FBECDBFDF91CF911F910F91089580E028
:10224000F3CFEF92FF921F93CF93DF9300D000D094
:1022500000D01F92CDB7DEB77C01FC0180810E94C7
:102260005C0D132F62E0C7010E94F810882381F0F3
:10227000812F86958695810F27960FB6F894DEBF3D
:102280000FBECDBFDF91CF911F91FF90EF900895CA
:1022900080E0F1CFFC0190819770673039F4923083
:1022A00018F081E0943039F480E00895643021F42E
:1022B00081E09130C9F308956A3029F4965081E0A5
:1022C0009230C8F3F1CF81E0F6CFFC01660F660FC4
:1022D000660F972F990F990F990F80818650823042
:1022E00020F084E0860F9C5F08958CEF860F945059
:1022F0000895DC01EC91EF70B4E0EB9FF001112444
:10230000E652F74F60817181828193810895CF9366
:10231000DF93FC012281DB01FFE02F9FA00DB11DA7
:102320001124FC01438154818C91880F880F880F00
:102330008C5F11969C911197990F990F990F9C5F43
:1023400057FD3DC030E0E32F3A3008F0E9E0EA0FF6
:10235000FB2FF11D2581622F62956695669563704E
:10236000623051F070E0EFEF633041F07FEF6130A9
:1023700021F470E0E1E002C071E0E0E02F73EA01D7
:10238000F8E02F9FC019D1091124D7FF1BC09A0173
:1023900063E0369527956A95E1F768EF6203D0010F
:1023A000639FB00D11244A0F5B1F220F220F220FD3
:1023B000240F2E9F800D1124279F900D1124DF9153
:1023C000CF910895220F220F220F2E9F800D1124EE
:1023D000279F900D11243F5FAE01B5CFFC01828194
:1023E0008A3078F4DF01A80FB11D15966C936F73D6
:1023F00023813481620F732F711D748363838F5F18
:1024000082830895FC01DC0115960F9621E02D933F
:102410008A179B07E1F710821182128214821382BD
:102420000895E92F572F262F30E0A82FB0E0681726
:1024300070F5CD01821B930B9C01852F90E06E2FD0
:1024400070E05E1738F5FB01E81BF90BCF0150E097
:102450004217530708F43DC048175907D0F1229F8F
:10246000B001239F700D700D1124889F9001899FEA
:10247000300D300D1124260F371F80E090E428170F
:10248000390758F49695879596958795F8CF2A1B26
:102490003B0BD3CF861B970BDACF70E060E0009741
:1024A00091F0FC01E60FF71F2E173F0728F02E1BB7
:1024B0003F0BBC016E0F7F1F96958795969587956C
:1024C00076956795ECCF81E04617570718F080E0C6
:1024D000089581E00895089590E080E008953F9286
:1024E0004F925F926F927F928F929F92AF92BF9224
:1024F000CF92DF92EF92FF920F931F93CF93DF93D0
:10250000CDB7DEB7E3970FB6F894DEBF0FBECDBFF1
:10251000909120069230B9F1F0F4992309F48BC11F
:10252000913009F4A7C0E3960FB6F894DEBF0FBE52
:10253000CDBFDF91CF911F910F91FF90EF90DF9072
:10254000CF90BF90AF909F908F907F906F905F9053
:102550004F903F900895943009F454C508F461C039
:10256000953009F7883011F08430E9F68091D00871
:10257000E0914D06F0E0EB52F74F9081981708F08C
:102580004CC580834AC5883009F04BC081E08093F8
:1025900020060091D1080F3030F61091D208173084
:1025A00010F6DD24D394D00EED2CF12C20E1129FF7
:1025B000C00111248E0D9F1D9C01220F331F820F1D
:1025C000931F825B994F0E94DB10882319F0D092F1
:1025D000D108A9CF1F5F40E1149F50011124C5010C
:1025E000800F911D9C01220F331F820F931F825B6E
:1025F000994F0E94DB10882319F01093D20893CFD3
:10260000EA0CFB1CC701880F991F8E0D9F1D825B72
:10261000994F0E94DB10882309F485CFD092D1080E
:10262000ECCF803209F160F4803109F07CCF8091E9
:10263000D208873008F086E08F5F8093D20873CF8E
:10264000803449F0803809F06ECF8091D208882319
:10265000A1F38150F2CF8091D1088F3008F08EE045
:102660008F5F8093D1085FCF8091D1088823C9F311
:102670008150F7CF8830A9F028F4843009F053CF87
:1026800082E0CAC0803209F4CCC0803409F04BCF5C
:102690008091D30890E001966DE070E00E945E2C7E
:1026A000C7C06091D308CE0101960E94830D898135
:1026B000811139CF6091D308683008F040C0CE0155
:1026C00001960E94830D89818130C9F18091D308E0
:1026D00057E0859FF0011124E95DFE4F448150E0F1
:1026E0002091CC083091CD082417350720F4909123
:1026F0004C06913021F5241B350B3093CD082093E7
:10270000CC082091D20870E1279F90011124E0911C
:10271000D1082E0F311DF901EE0FFF1FE20FF31F3D
:10272000E25BF94F9EE09083877081838FEF828315
:1027300082E0809320061092D3080E947C0FF090D4
:10274000D3088AE0F81609F44EC08F1508F445C086
:1027500098E0F91608F4E7CE0091D208E0E10E9F68
:1027600080011124C090D108C00ED12ED11C860149
:10277000000F111FF801EC0DFD1DE15BF94FE0802A
:102780008E2D0E945C0D862F90E0880F991F63E0CC
:1027900070E00E945E2C8091CC089091CD08861745
:1027A000970728F480914C06813009F0BCCEF8E000
:1027B00080E8FF1280E40C0D1D1DF801E05EF94F6A
:1027C000E82AE7A68091CC089091CD08861B970B4C
:1027D0009093CD088093CC08A6CEABE0FA1639F0E2
:1027E000BCE0FB12A0CE84E0809320069CCE8091BA
:1027F0004006909141066091D00870E0DC01ED91B7
:10280000FC910190F081E02D08EC18E02EEC37E00F
:1028100041E256E0099583E0809320061092D308A8
:1028200082CE8091D308882311F0815001C08CE0C2
:102830008093D30878CE803209F48CC0803409F4B8
:1028400082C0883009F06FCE1091D308153008F09F
:10285000CFC31092C9081092C8081092CD081092E8
:10286000CC081092D0081092CF081092CE08CE015A
:1028700085960E940212CE0101960E9402121092C9
:102880003F06123009F490C108F06AC0113009F413
:10289000FDC081E08DA38EA365E8CE0185960E94E0
:1028A000EE1162E4CE0185960E94EE1165E0CE0144
:1028B00085960E94EE1168E4CE0185960E94EE1185
:1028C00062E8CE0185960E94EE1165ECCE018596F8
:1028D0000E94EE1163E8CE0185960E94EE1167E436
:1028E000CE0185960E94EE1165E0CE0185960E948C
:1028F000EE11ADA0BEA0CFA0D8A4E9A4FAA40BA568
:102900001CA52DA53EA54FA558A969A97AA98BA9F3
:102910000E94150584E1809342068AE08093430675
:1029200084E496E09093410680934006E0E2F6E06E
:1029300080E09FEF3396803809F44CC213A614A6AA
:1029400095A78F5FF7CF8091D30890E0019666E05E
:1029500070E0A4CE8091D308811167CF85E068CF65
:10296000133009F4A2C1143009F093CF1DA31EA3A4
:1029700062E0CE0185960E94EE1163ECCE01859651
:102980000E94EE1164E8CE0185960E94EE1165E486
:10299000CE0185960E94EE1165E0CE0185960E94DB
:1029A000EE1162E4CE0185960E94EE1165E8CE013B
:1029B00085960E94EE1163E4CE0185960E94EE1189
:1029C00065E0CE0185960E94EE1163E4CE01859606
:1029D0000E94EE118DE0898386E08A8363E0CE0158
:1029E00001960E94EE1165ECCE0101960E94EE1157
:1029F00063E8CE0101960E94EE1162ECCE010196D1
:102A00000E94EE1163E0CE0101960E94EE1161EC8E
:102A1000CE0101960E94EE1162E0CE0101960E9465
:102A2000EE1163ECCE0101960E94EE1163E8CE0137
:102A300001960E94EE11ADA0BEA0CFA0D8A4E9A43B
:102A4000FAA40BA51CA52DA53EA54FA558A969A9BB
:102A50007AA98BA90E941505A980BA80CB80DC8059
:102A6000ED80FE800F81188529853A854B855C8530
:102A70006D857E858F850E9415058EE180934206C7
:102A800086E1809343068AE496E04CCF11E01DA3D3
:102A90001EA362E8CE0185960E94EE1167E4CE0186
:102AA00085960E94EE1161E8CE0185960E94EE1196
:102AB00062E4CE0185960E94EE1162E8CE01859611
:102AC0000E94EE1164E4CE0185960E94EE1163E04F
:102AD000CE0185960E94EE1162ECCE0185960E9491
:102AE000EE1162E0CE0185960E94EE1164ECCE01FB
:102AF00085960E94EE11198386E08A8363E0CE01F9
:102B000001960E94EE1163E4CE0101960E94EE113F
:102B100062E8CE0101960E94EE1161E4CE010196B9
:102B20000E94EE1161E8CE0101960E94EE1169E467
:102B3000CE0101960E94EE1163E0CE0101960E9443
:102B4000EE1162ECCE0101960E94EE1162E0CE0120
:102B500001960E94EE1164ECCE0101960E94EE11E6
:102B6000ADA0BEA0CFA0D8A4E9A4FAA40BA51CA533
:102B70002DA53EA54FA558A969A97AA98BA90E94A0
:102B80001505A980BA80CB80DC80ED80FE800F81A6
:102B9000188529853A854B855C856D857E858F8571
:102BA0000E94150589E1B7CE11E01DA31EA365E8BB
:102BB000CE0185960E94EE1162E4CE0185960E94B8
:102BC000EE1162E0CE0185960E94EE1162E4CE0124
:102BD00085960E94EE1162E8CE0185960E94EE1164
:102BE00063E4CE0185960E94EE1163E0CE018596E6
:102BF0000E94EE1162ECCE0185960E94EE1162E019
:102C0000CE0185960E94EE1163ECCE0185960E945E
:102C1000EE118EE089831A8364ECCE0101960E9446
:102C2000EE1165E8CE0101960E94EE1162E4CE013C
:102C300001960E94EE1163E0CE0101960E94EE1112
:102C400062E4CE0101960E94EE1163E8CE01019686
:102C50000E94EE11ADA0BEA0CFA0D8A4E9A4FAA412
:102C60000BA51CA52DA53EA54FA558A969A97AA914
:102C70008BA90E941505A980BA80CB80DC80ED80ED
:102C8000FE800F81188529853A854B855C856D8589
:102C90007E858F850E94150584E1809342068AE037
:102CA0008093430686E496E03DCE02E00DA317E054
:102CB0001EA362E0CE0185960E94EE116CE4CE0167
:102CC00085960E94EE1162E8CE0185960E94EE1173
:102CD00067ECCE0185960E94EE1166E0CE018596E6
:102CE0000E94EE1162ECCE0185960E94EE1162E820
:102CF000CE0185960E94EE1164ECCE0185960E946D
:102D0000EE1161E0CE0185960E94EE1163E4CE01E2
:102D100085960E94EE1109831A8362E0CE01019626
:102D20000E94EE116CE4CE0101960E94EE1162E861
:102D3000CE0101960E94EE1167ECCE0101960E9431
:102D4000EE1166E0CE0101960E94EE1162E4CE0122
:102D500001960E94EE1162E8CE0101960E94EE11EA
:102D600064E4CE0101960E94EE1161E0CE0101966D
:102D70000E94EE1163ECCE0101960E94EE11ADA00F
:102D8000BEA0CFA0D8A4E9A4FAA40BA51CA52DA58C
:102D90003EA54FA558A969A97AA98BA90E94150536
:102DA000A980BA80CB80DC80ED80FE800F81188501
:102DB00029853A854B855C856D857E858F850E944A
:102DC00015058AE08093420688E08093430688E4F4
:102DD00096E0A8CD30E055245394BFE06B2E8824B4
:102DE0008A9412E0412E80913F06381708F0DEC029
:102DF000832F311181E0869D7001112487010F5DC1
:102E0000194FF8019081218140E071E0D8011296BC
:102E10008C911297481708F0A3C0E42F4A3008F0AD
:102E2000E9E0EE0DFF2DF11DEA5DF94FE0818E2FF7
:102E30008295869586958370823051F050E06FEFD1
:102E4000833041F050E061E0813021F05FEF01C05C
:102E500051E060E07111782EEF739E2E322EB92E64
:102E6000A12CB0E13B9E60011124CB0CD11C9A1423
:102E700009F46DC0F601EE0FFF1FDF01AC0DBD1DA3
:102E8000A05EB94F9E96BC91882309F45AC072E0A7
:102E9000771669F0AB2FAB7FA33049F0B53039F02E
:102EA000A5EFAB0FA23018F070E0BD3009F478E068
:102EB000813081F0A3E07A1669F0ACEFAB0FA3305C
:102EC00048F0A7EFAB0FA23028F0BC3019F0A0E01B
:102ED000BD3009F4A4E07A2B823069F0772059F0F4
:102EE000B33049F0B63039F0A8EFAB0FA43018F08A
:102EF000A0E0BD3009F4A2E07A2BA1E0833069F0B4
:102F00007A1609F1B430F9F0A9EFAB0FA230D8F07E
:102F1000BA50A1E0B43008F0A0E0A72BA350AD3028
:102F2000A0F4B0E0A65EBE4FAC91EC0DFD1DE25BDF
:102F3000F94FA08311828282A394B60E350E782EAB
:102F400090CF78E0B7CFA1E0E8CFA0E0EECF969E9B
:102F5000900D1124959E200D11244F5F70E056CFE7
:102F6000F8014181F0E14F9FA0011124EC914E0F37
:102F7000511DFA01EE0FFF1FE40FF51FE25BF94F41
:102F8000508211828282B0E12B9FF0011124AF01A7
:102F9000490F511DFA01EE0FFF1FE40FF51FE25B11
:102FA000F94F4082118282823F5F1DCF8091D3080A
:102FB00080934D061092D0088091430690E0909344
:102FC000CD088093CC088091420690E09093CF0882
:102FD0008093CE0888E08093D10884E08093D20863
:102FE0001092D30890E080E00E94A82B82E0FCCBF6
:102FF000153009F098CA8091D40891E08927809310
:10300000D40891CA843011F481E0EECB883009F005
:103010008ACA8091D3088C3019F410922006FECB16
:103020008A3009F080CA0091D20850E1059FF00172
:1030300011240091D1080E0F1F2F111DF801EE0F62
:10304000FF1F0E0F1F1FF801E15BF94F80810E94E7
:103050005C0D66958091CC089091CD08680F792F12
:10306000711D7093CD086093CC08F801E25BF94FB5
:10307000108211828FEF828385E08093CB0580E4FC
:10308000809390008CE195E1909399008093980053
:10309000ADCFCF93DF93C82FD62F8091A8018C237B
:1030A00039F48091A9018C2319F08C2F0E946F12A2
:1030B000DD23D9F08C2F0E944C098823C9F0809120
:1030C000000181110FC080919E0190919F0166E0E7
:1030D00070E00E944A2C892B41F48C2FDF91CF9114
:1030E0000C946F12815080930001DF91CF9108956D
:1030F0008091A8018C23C9F38091A901C823A9F765
:1031000084E1F1CF1F93CF93DF93EC0182E08093B2
:10311000CB0580E48093900084E59DE09093990036
:10312000809398001981129516951695137021F0C9
:1031300088818F70863029F41982DF91CF911F9199
:103140000895CE010E9479117F73115020E4129FDF
:10315000C0011124872B898386EF9FEF9C838B838B
:10316000ECCF8F929F92AF92BF920F931F93CF930A
:10317000DF93CDB7DEB7A1970FB6F894DEBF0FBED1
:10318000CDBF19A2423008F44AE08E010F5D1F4FF7
:10319000842E912CB12CA12CA50194010E940D2C00
:1031A000E62FB901CA01EA3044F5E05DD801EE939B
:1031B0008D01232B242B252B79F790E080E01097AD
:1031C00069F0FD0101900020E9F73197AF014A1B3A
:1031D0005B0BBD018CE196E00E940909A1960FB638
:1031E000F894DEBF0FBECDBFDF91CF911F910F913D
:1031F000BF90AF909F908F900895E95CD7CFFC016E
:1032000001900020E9F73197AF01481B590BBC0131
:103210008CE196E00C9409092F923F924F925F92B5
:103220006F927F928F929F92AF92BF92CF92DF92D6
:10323000EF92FF920F931F93CF93DF93CDB7DEB73B
:10324000C457D1090FB6F894DEBF0FBECDBF40E220
:1032500056E0E1965FAF4EAFE1972A01B12CA12C69
:10326000AF961FAEAF97AE961FAEAE97F12C5FEF45
:10327000A8965FAFA897150188E0281A3108620167
:10328000912C812C10E0D6019E968C918E3029F5E0
:10329000F60186A58E3009F40EC1E091D30827E02F
:1032A0002E9FF0011124E95DFE4FDE01119687E0AB
:1032B00001900D928A95E1F74A81A8964FAFA897A1
:1032C000612F7F2DCE0101960E946511AF968FAFC1
:1032D000AF97AE969FAFAE97F8C080912006813031
:1032E00009F58091D10881131DC08091D2088F11FA
:1032F00019C06091D3086830A8F48091CA089091F1
:10330000CB0823E0969587952A95E1F78370992756
:10331000892B41F0CE0101960E94830D898188237B
:1033200009F4B6CFD6019E964C91B8E04B9FA00110
:1033300011244A595E4FEE24E39408E028E0B501D9
:10334000C4010E945A091F5F53E0C50ED11C88E0DA
:10335000880E911C103109F096CFF39498E0A90ED5
:10336000B11CA0E34A0E511CB0E4AB16B10409F045
:1033700082CFAB961FAEAB97E196EEADFFADE19776
:10338000A796FFAFEEAFA797AA961FAEAA97A796EC
:10339000AEADBFADA7979E968C919E978E3009F0EB
:1033A00022C1D096EC91EF3F09F41DC1B5E0BE9F5C
:1033B000F0011124E253F84FDE01959685E001906B
:1033C0000D928A95E1F78EA18F7309F40CC161E229
:1033D00076E0CE0185960E9487114C01A796EEAD4E
:1033E000FFADA79787A5482F50E003E05595479577
:1033F0000A95E1F7142F1770FCE01F9FF02D1124A0
:10340000A996FFAFA9970E945C0D29833A834B834D
:103410005C836D837E838F83AA966FADAA97AB96EC
:103420007FADAB97CE0101960E9465113C01E82C5F
:10343000F12CC82ED12C27014C185D08A9962FAD70
:10344000A997E22FF0E04E9EC0014F9E900D5E9E28
:10345000900D112464E670E00E945E2C062D060F8C
:10346000292D30E0A72CB12C19012A183B082E9EDB
:10347000C0012F9E900D3E9E900D112464E670E0D9
:103480000E945E2C472D460FA796AEADBFADA79705
:103490009F96EC91E770E150E73008F08DC0F0E0C6
:1034A000EC5AF54E0C94722C621B711BCB1B9B1BB0
:1034B000C31BE81BAF1A87A50E945C0D29833A83C2
:1034C0004B835C836D837E838F8389818630A8F0F4
:1034D000863089F480E0D6019F962C91221F222706
:1034E000221F280F02E043ED57E0B101C401089705
:1034F0000E94930528CF82E0EECF712C612C962D8F
:10350000662061F0F60187A5282F30E0913021F187
:1035100080E490E082239323892BB1F48981A30175
:1035200093E0440F551F9A95E1F7F8E18F9F400D06
:10353000511D11244C5B564FEE24E39408E028E023
:10354000B501C4010E945A092FEF621A720A43E0C2
:1035500064167104A1F6F7CE80E890E0DBCFE12E8F
:10356000F12CC70101966C01CC0CDD1CC80ED91ED4
:10357000712CB2E0EB0EF11CE42FE250FF0B5F0167
:10358000402F4250550B4A017C141D0464F50E94E3
:10359000A32BB7010E945E2C8501080F191F0E9402
:1035A000A32BB7010E945E2C40E0B801880D991D45
:1035B0000E942F0A7394E8CF861418F426014E183F
:1035C0005F08971418F41501221A330A642F70E06B
:1035D000802F90E0241435040CF06FC0403418F4B0
:1035E00042E00E945A05AA969FADAA979F5FAA96AD
:1035F0009FAFAA97A796AEADBFADA7971396A79614
:10360000BFAFAEAFA797903109F0C1CEAB96BFADBB
:10361000AB97BF5FAB96BFAFAB97E196EEADFFAD9B
:10362000E197F096E196FFAFEEAFE197B83009F081
:10363000A3CEF12C75E0E72EE2E0CE2ED12C8091C6
:10364000C8089091C908F816190608F040C1FE9CF8
:10365000800111240253184FD80113968D919C912B
:10366000149797FD28C011968C918F7321F161E218
:1036700076E0C8010E948711B82EA92EC8010E94C9
:103680007911262FF80183819481959587959595D9
:103690008795B6010E945E2C4A2D4450550BBA0105
:1036A000680F711D03E044EB50E0AB2DA450BB0B41
:1036B000CD010E949305F394C2CF20E042E00E9426
:1036C000210C91CFE42EF12C10E020E042E0B70174
:1036D000C80101970E94210C20E042E0B701C80117
:1036E000EECFE42EF12C10E040E0B701C8010E94BB
:1036F0002F0A57015FEFA51AB50A68018FEFC81AA4
:10370000D80A40E0B501C6010E942F0A01501109F4
:1037100040E0B501C8010E942F0A91E0E91AF108C2
:1037200040E0B701C6010E942F0A40E0B701C8017E
:103730000E942F0A58CFE02FF0E0842E912CA81879
:10374000B908A9E1AA9DC001AB9D900D112464E6C2
:1037500070E00E945E2CE42EE60E2E2D30E0CE1A94
:10376000DF0AB9E1BC9DC001BD9D900D112464E646
:1037700070E00E945E2C060F402F50E0B401CF0194
:103780000E94120B30CF642F70E041E0802F90E058
:103790000E944A0A28CFA996EFADA997E23308F014
:1037A00022CF8091CA089091CB08AC014370552775
:1037B000240F351F2150310963E070E00E944A2C2C
:1037C000AC014E0D5F1D41505109B501C601D8CF66
:1037D000169581E0810F242E312CA02EB12C082FBC
:1037E00010E0482F440F4F5FB101601B710B20E0C8
:1037F000C5010E94210CCC24C394D12CC01AD10A3B
:10380000712C612C601A710A660C771CEE24E3940B
:10381000F12C912C812CE396BFAEAEAEE397E596EA
:103820003FAE2EAEE597D7FC07C001501109F2E07C
:103830006F0E711CC60CD71C2FEF821A920A42E041
:10384000E40EF11CCE0CDF1C502E550C5394A9969F
:103850005FAEA99720E0452D2101401A510AB2011F
:10386000E3968EAD9FADE397880D991D0E94210CC4
:10387000E5968EAD9FADE59788199909AD969FAFF6
:103880008EAFAD9720E04E2DBC01C501800F911F7A
:103890000E94210C20E0A9964FADA997B201E396B2
:1038A0008EAD9FADE397881999090E94210C20E005
:1038B0004E2DAD966EAD7FADAD97C501801B910BC2
:1038C0000E94210C801691060CF4ADCF8CCEC090D6
:1038D000D208CC0CCC0CCC0CA090D108AA0CAA0C11
:1038E000AA0CD12CB12C28E048E0B601C5010E94F9
:1038F0004A0C912C812C53E0E52EF12C8501095FB7
:103900001F4F1601B7E02B0E311C3501E8E06E0E9B
:10391000711C2601F8E04F0E511C8091CA0890914D
:10392000CB0843E0969587954A95E1F7880D991D58
:10393000B7010E944A2C892BE1F441E0B601C50190
:10394000880D991D0E942F0A41E0B601680D791D6E
:10395000C8010E942F0A41E0B101C30188199909E9
:103960000E942F0A41E0B20168197909C5010E943D
:103970002F0A2FEF821A920A48E08416910469F602
:1039800080912006813039F480912006813009F041
:1039900065C001E068C084E00E944C098823A1F35F
:1039A00080912006833009F0C1C088E00E944C0954
:1039B000882309F4BBC0B12C35E0A32E8B2D90E0F9
:1039C0002091C8083091C9088217930708F0AEC04B
:1039D000A89EF001A99EF00D1124E253F84FDE01DC
:1039E00011968A2D01900D928A95E1F78C819D8127
:1039F00097FD32C08A818F7379F161E276E0CE0162
:103A000001960E948711C82EE92ECE0101960E94D0
:103A10007911972E1A81F12CD12CB70166507109BA
:103A200001E023E046E0C60103970E947A0C55E0CE
:103A3000E51AF10880E4E816F10470F41F731A9D8A
:103A4000C0011124692D70E00E944A2C462FB70155
:103A5000C60102970E945A05B394B0CF8091D20854
:103A600008E3811196CF1092020181E08093A301B7
:103A700010E081E090E09093A5018093A401109361
:103A8000A7010093A60164E28CE196E00E94960BE8
:103A900080914C06813009F03FC061E28CE196E0F4
:103AA0000E94960B61E28CE196E00E94960B61E227
:103AB0008CE196E00E94960B89E290E09093A5013C
:103AC0008093A4011093A7010093A6016CE48CE1FC
:103AD00096E00E94960B6091CE087091CF0890E01E
:103AE00080E04AE00E94B11889E590E09093A5013A
:103AF0008093A4011093A7010093A60162E58CE1D5
:103B000096E00E94960B6091D00870E090E080E013
:103B10004AE00E94B11844CF6091CC087091CD0862
:103B200090E080E04AE00E94B118C6CF8091200664
:103B3000813009F046C18091D208A0E18A9FC0017E
:103B400011240091D108800F911D8C01000F111FCD
:103B5000080F191FF801E05EF94F86A58E3009F0B5
:103B600030C1015B194FC8010E942111A8968FAF87
:103B7000A89764E0C8010E94F810D82E8091CA0866
:103B800083FD48C08091D308883051F18091D308DB
:103B9000893071F469E0CE0101960E94830D89811C
:103BA000811106C0D8018C910E945C0D823031F1E8
:103BB0008091D308883009F4F2C08091D30889300D
:103BC00049F569E0CE0101960E94830D898181113A
:103BD00021C0D8018C910E945C0D8430D9F4EEC0D4
:103BE00068E0CE0185960E94830D8DA18111CECF14
:103BF000F80180810E945C0D723041F6A8968FAD6D
:103C0000A89786958695A896FFADA897F80FA896D1
:103C1000FFAFA897F80180810E945C0D29833A8349
:103C20004B835C836D837E838F836091D108709119
:103C3000D208CE0101960E946511AF968FAFAF9763
:103C4000AE969FAFAE97A896FFADA897FF3FD1F075
:103C5000AE962FADAE97022F10E0AF964FADAF9757
:103C6000E42EF12C4F2FB801C7010E944A0ADD2033
:103C700049F0B8016C50710928E148E1C7010C977F
:103C80000E944A0C80912006813009F06EC001E04C
:103C900029E040E867E370E090E080E00E947A0C61
:103CA00040E867E370E090E080E00E945A05D12C84
:103CB000C12C10E0AA24A394B12C9FE2892E912C50
:103CC000612FCE0101960E94830D8981823009F413
:103CD0004CC08091D308811376C04A815B81E12C6E
:103CE00008E028E068E370E0C6010E945A09B0923B
:103CF000A501A092A4019092A7018092A601CE01F5
:103D000005960E94FF188C818823D9F060E28CE12F
:103D100096E00E94960B68E28CE196E00E94960B7A
:103D200064E28CE196E00E94960B6C8170E090E07A
:103D300080E04AE00E94B11869E28CE196E00E94BE
:103D4000960B8981813051F4E12C08E028E04CEA9F
:103D500050E068E370E0C6010E945A091F5F58E016
:103D6000C50ED11C103109F0ABCFCC58DF4F0FB6C8
:103D7000F894DEBF0FBECDBFDF91CF911F910F91A1
:103D8000FF90EF90DF90CF90BF90AF909F908F907B
:103D90007F906F905F904F903F902F90089568E0D4
:103DA000CE0185960E94830D8DA1811106CFF80169
:103DB00080810E945C0D743009F0FFCEDD24D39425
:103DC00029CFD12C40CF00E028E048E068E370E044
:103DD000C6010E947A0C4A815B81EE24E39408E0DC
:103DE00028E068E370E0C6010E945A09AACF9F92BA
:103DF000AF92BF92CF92DF92EF92FF920F931F93F9
:103E0000CF93DF9300D000D000D01F92CDB7DEB7A4
:103E10007C018B015A01922EFB0160816F700E9420
:103E20004A11D82E882309F459C0F7018081877080
:103E3000823091F063E0C7010E94F810D82E8823E9
:103E400059F00E94A32B63E070E00E945E2CDD24F9
:103E5000D394892B09F0D12CF70180810E945C0D4D
:103E6000C52E60E0C7010E94F810882309F448C0FD
:103E70008C2D8695C80E8C2D90E061E070E0992025
:103E800011F062E070E00E945E2CF8018181982FB1
:103E90009F736917B8F1C8010E948218C8010E9477
:103EA0007911F50120813181290F311D3183208362
:103EB0008FEFF7018183F70180818770863071F47D
:103EC0000E94A32B6AE070E00E945E2C892B31F4E3
:103ED000F801838194810A979483838327960FB690
:103EE000F894DEBF0FBECDBFDF91CF911F910F9130
:103EF000FF90EF90DF90CF90BF90AF909F9008958C
:103F000080E0B8CF961B9F73807C892B8183DD2056
:103F100091F280818F702FE0833009F427E0F0E187
:103F20002F9F90011124822BF8018083C4CFFF9230
:103F30000F931F93CF93DF93EC01F62E0881198125
:103F4000C8010E94B32BF81621F06F2DC8010E9402
:103F5000CD2BCE01DF91CF911F910F91FF9008954E
:103F60001F920F920FB60F9211248F939F938091FF
:103F7000E1009091E100937F9093E10083FF0FC0F7
:103F80001092E90091E09093EB001092EC0092E324
:103F90009093ED001092CA0198E09093F00082FF98
:103FA00022C093E09093E9009091F200992319F0D8
:103FB0009AE39093E8009091BB01992341F090918E
:103FC000BB0191509093BB01911101C05D9A9091FA
:103FD000C901992341F09091C90191509093C90171
:103FE000911101C0289A84FF18C08091E2008E7E52
:103FF00081608093E2008091E1008F7E8093E100F8
:104000008091BC018E7E80618093BC019F918F91D5
:104010000F900FBE0F901F90189580FFF7CF8091E3
:10402000E2008E7E80618093E2008091E1008E7ECE
:104030008093E1008091BC018E7E8160E5CF1F926C
:104040000F920FB60F921124CF92DF92EF92FF9250
:104050000F931F932F933F934F935F936F937F9390
:104060008F939F93AF93BF93EF93FF93CF93DF9380
:10407000CDB7DEB76C97DEBFCDBF1092E90080915F
:10408000E80083FF25C068E0CE0145960E944D08F8
:1040900082EF8093E8008D8987FF39C09091E80016
:1040A00090FFFCCF982F907609F034C19E894F89FC
:1040B000588D2F89F88C911131C0803861F580912D
:1040C000BA018093F1001092F1008EEF8093E80026
:1040D0006C960FB6F894DEBF0FBECDBFDF91CF91C7
:1040E000FF91EF91BF91AF919F918F917F916F91D0
:1040F0005F914F913F912F911F910F91FF90EF9002
:10410000DF90CF900F900FBE0F901F9018959EEFED
:104110009093E800C7CF1092F100D5CF913059F4B9
:104120008111D3CF4130510581F68091BA018D7F45
:104130008093BA01CACF933049F48111C6CF413080
:10414000510519F68091BA018260F2CF953041F4A1
:104150008091E80080FFFCCF20682093E300B5CF7A
:10416000963009F0A9C00B8D1C8D22E01092E90059
:104170001092B8011092B701F2122EC01092B6013F
:104180001092B5010E941C081F8299E09983FA825F
:1041900091E09E8390EA98879AEF99872091B701E2
:1041A0003091B801275F3F4F3C832B838D83109262
:1041B000E9001092B8011092B7011093B601009374
:1041C000B50149E050E0BE016F5F7F4F80E00E9483
:1041D000F6070E941C0879CF1093B6010093B50131
:1041E0000E943307DC0112960D911C9101151105F7
:1041F00009F451C1D801ED91FC910480F581E02DC5
:10420000BE016B5E7F4FC8010995009709F03EC162
:10421000F80100851185EACFF3E0FF120EC08F8907
:10422000882309F440C0823061F440E867E084E00C
:1042300099E00E949B22811148CF81E28093EB009C
:1042400047CF813029F440E86BE088EF98E0F1CF68
:10425000833099F70E943307DC011296ED90FC90B1
:104260008E010F5F1F4F6801E114F10479F0D7014F
:10427000ED91FC910680F781E02DB801C701099509
:10428000080F111DF701E084F184EECFD8011C92D4
:10429000F60101900020E9F73197BF016C197D0903
:1042A00040E0C601C6CF62EE78E0FB01449150E0E9
:1042B00080E80E94F60709CF973009F4BECF983006
:1042C00021F481E08093F10000CF993009F0FDCE18
:1042D000837009F0B2CFE4E1F1E081E031E096E3F0
:1042E0002191222371F08093E9003093EB00DF01EC
:1042F00011972C912093EC009093ED008F5F873005
:1043000079F78EE78093EA001092EA008F89809314
:10431000CA01DBCE8B8D9C8D1092E9001092B80102
:104320001092B7019093B6018093B501898D8111E8
:1043300092C08E899D89913A49F4813209F07DCFEE
:1043400047E050E067E071E080E0B3CF913209F0E0
:1043500074CF833269F48F89988DB0E0A0E08093A8
:10436000030190930401A0930501B0930601ADCE23
:10437000803269F48091E80082FFFCCF67E087E03B
:1043800091E00E944D088BEF8093E8009ECE823230
:1043900009F09BCE8F8980930E01EEEFFFE78591A8
:1043A00094918B3F9C4D51F1E0E0F8E08091070142
:1043B00090910801A0910901B0910A01803B9440BD
:1043C000A105B105F1F480910E0180FD1AC0EE3F08
:1043D0008AE0F80789F587E797E7918380838091E2
:1043E00060008093B90188E19BE00FB6F894A8952E
:1043F000809360000FBE9093600067CEEEEFFAE00E
:10440000D5CF808191818737974709F05ECEA895F7
:10441000809160008861809360008091B9018093F1
:104420006000EE3F2AE0F20789F08091FE0A909149
:10443000FF0A9183808349CE8081918187379807D5
:1044400051F29093FF0A8093FE0AC5CF1092FF0AA3
:104450001092FE0A3ACE0E943307DC0112960D91AB
:104460001C910115110509F4E8CED801ED91FC91DC
:104470000190F081E02DBE016B5E7F4FC801099570
:10448000811123CEF80100851185EBCF181619068E
:104490000CF41BCED2CEF1E0FF12BECE66EE78E079
:1044A00004CF0F920FB68F939F93EF93FF9380915A
:1044B000AC018D5F8D3708F08D578093AC01EDEA2C
:1044C000F1E080818E4F808391819F4F9183828123
:1044D0008F4F828383818F4F8383E1EBF1E0808173
:1044E0008F5F808381818F4F818382818F4F828311
:1044F00083818F4F83838FB18F6066991C9B882740
:104500008F3681F48091AB01981B963068F0E0E023
:10451000F8E087E78083818388E180936000F093EF
:104520006000FFCF9093AB01FF91EF919F918F912E
:104530000FBE0F901895EF92FF920F931F93CF939A
:10454000DF93F82E192FE62E042F81E0860F880FB7
:104550000E94C80783E00E94C807CF2DD12FEC0E20
:10456000FD2EF11CCE15DF05B9F007FF13C0FE01CB
:1045700084910E94C807182F80E00E94C8078123F9
:1045800021968111EFCFDF91CF911F910F91FF9075
:10459000EF9008958881EDCF81E0F5CFCF93DF9341
:1045A0001092CF051092CE0588EE93E0A0E0B0E027
:1045B0008093D0059093D105A093D205B093D305F5
:1045C00083E691E09093CD058093CC058FEF9FEF2C
:1045D0009093D9058093D8051092DA0847E040936C
:1045E000DB0892E09093DC0881E08093DD08809303
:1045F000DE0838E03093DF088093E0088093E1081C
:104600009093E2082CE02093E3089093E4088093D1
:10461000E50823E02093E608C4E1C093E7089093FF
:10462000E8088093E90854E05093EA086DE060934D
:10463000EB088093EC088093ED0865E06093EE084A
:104640006BE26093EF085093F0089093F10856E006
:104650005093F208C093F3089093F4089093F508F0
:104660004093F6084EE14093F7082093F8089093A2
:10467000F9083093FA083AE33093FB089093FC086A
:104680002093FD0899E09093FE089FE39093FF0824
:104690008093000920930109DAE0D09302099093F6
:1046A0000309809304092093050981E296E00E94A2
:1046B000021280E396E00E94021210923F061092CE
:1046C000410610924006C0934206D093430687E805
:1046D00091E0909345068093440681E891E09093A1
:1046E0004706809346068BE791E0909349068093B6
:1046F000480685E791E090934B0680934A06EEE4E6
:10470000F6E08FEF108211828283339697E0EE3CC1
:10471000F907C1F7E0E2F6E080E09FEF33968038DA
:1047200029F013A614A695A78F5FF8CFEEECF7E05B
:1047300087E412821482138281831082359698E076
:10474000E83CF907B1F71092D1081092D208109204
:1047500020061092CB081092CA081092C908109235
:10476000C8081092D30810924C061092D4081092E8
:10477000D5081092D6081092D7081092D808109237
:10478000D90810924D0610921F0610921E068DE851
:1047900091E090931D0680931C06DF91CF910895C0
:1047A000CDB7DEB7EB97DEBFCDBF789483E084BD95
:1047B00083E085BD81E080936E00E1E8F0E083E076
:1047C0008083E0E881E08083E1E983E08083E0E9C1
:1047D00081E08083E1EC87E08083E3EC81E080830B
:1047E000E0EC82E08083E2EC81E08083EAE787E02E
:1047F0008083806880831092CA011092BA0110925F
:10480000BC018091D70081608093D70080EA8093BB
:10481000D80089B5806189BD89B5826089BD09B438
:1048200000FEFDCF81E090E00E945A088091D80000
:104830008F7C80618093D8008091E000807F80939E
:10484000E0008091E1008E7E8093E1008DE0809316
:10485000E200559A209A81EC80937C0081E785B92B
:1048600087E684B985E38BB98FE38AB9769A6E9827
:1048700080EF81BB10BA80E58CBD81E08DBD85E005
:104880000E943609599A85E00E9436095C98E6E84C
:10489000F7E085918EBD00000DB407FEFDCFE33932
:1048A000C1F75C9A81E88093640081E080936500A1
:1048B0000E94570980E80E944C09882369F15C989E
:1048C00085EA8EBD00000DB407FEFDCF5C9A2E98E0
:1048D00058982D988091640080628093640081E0F4
:1048E00083BF889513BEFCCF2D9A88EC0E943609B1
:1048F00058986FEF82E090E00E94BB2B84EF91E02C
:104900000E945A08589A84E80E944C098111FBCFF2
:104910000EC088EC0E94360984E00E944C0988236E
:1049200001F12D9884E80E944C098111DDCF84E1CA
:104930000E944C09882369F32D9A88EC0E9436095D
:104940002E9860E082E090E00E94BB2B84EF91E023
:104950000E945A082E9A84E10E944C098111FBCFD3
:10496000D8CF2D9A82E090E00E94B32B882309F4DF
:104970005DC00E94460981E090E00E94B32B182F91
:10498000147081FF0EC011112E98E1EFCE2EDD24A0
:10499000DA9480E40E944C09882309F44AC02E9AD4
:1049A000589A82E30E9436090E9439098111F9CF91
:1049B0008091A2018093D408109290008AE08093A5
:1049C00091000E94DC061092A7011092A60110929D
:1049D000A5011092A40180E1809301018AEC90E08E
:1049E0000E94B32B0BEC10E08F3509F07FC075ED02
:1049F000E72E78E0F72E0BEC10E0C8010E94B32BF5
:104A0000D7018D937D010F5F1F4F003D1105A9F761
:104A10008091A001882309F47FC01092A00180E05A
:104A200090E0892BA9F30E940000F2CF0E94410977
:104A3000A2CF112331F024E0C216D10411F42E9A32
:104A4000589881E00E94E906EE24E39400E128E50D
:104A500046ED56E0B60184E190E00E945A090E94BA
:104A600057098FE00E9436093FEFC31AD30A49E184
:104A7000C416D10409F08DCF112311F0589A2D9846
:104A800080E991E00E945A082D9A81E090E00E940E
:104A9000B32B80FF86CF8AE090E00E94B32B9FEF7C
:104AA000980F9E3F08F07DCF22E330E03093A501C0
:104AB0002093A40128E330E03093A7012093A601BE
:104AC0000AE010E0682F8CE196E00E94960B0F5FE1
:104AD0001F4FC8010E94B32B0031110599F70E94A6
:104AE000570988EE93E00E945A085BCF1A83098326
:104AF00060E0CE0101960E94971F0F5F1F4F003D9F
:104B00001105A1F78AEC90E09A8389836FE5CE01C5
:104B100001960E94971F7CCF9091AD018091A101D9
:104B2000B92FB81B8B2F20910101B21748F48F5F6A
:104B3000821708F074CF81E083BF889513BE6FCFD2
:104B400081E08093A0019093A101EEE9F1E08081E2
:104B500091810196808391838091CB05882339F0E0
:104B600081508093CB05811102C0109290008091FA
:104B7000A9018093A8010E9439098093A90160E0EE
:104B800088E00E94491860E084E00E94491861E0D2
:104B900080E20E94491861E080E40E94491861E0C7
:104BA00080E80E94491861E080E10E94491880E88D
:104BB0000E944C09882351F084E00E944C0988230C
:104BC00029F080E10E944C0980934C0680912006D8
:104BD000833051F488E00E944C09882329F084E056
:104BE0000E944C09811117C1E1E0EFA71BA605E067
:104BF0008091CA089091CB0801969093CB0880933E
:104C0000CA0880912006833009F0F2C310E04FE01B
:104C1000742E50E4652E6CE1862E65E1962EC12E31
:104C2000D12C8091C8089091C908C816D90608F0FF
:104C30008FC0109FC00111249C012253384F79016D
:104C4000A090CA08B090CB08D90111968C918F73AF
:104C500001F1C9010E947911F701908192959F702D
:104C600060E009F06FE0860F682F70E0660F771F35
:104C7000C5010E944A2C892B61F40C9DF0010D9D09
:104C8000F00D1124EF52F84F8081918101969183AC
:104C90008083C50163E070E00E944A2C892B79F47F
:104CA000D7018C91282F22952F7049F02150B0E127
:104CB0002B9F900111248F70822BF7018083D701E5
:104CC00011968C9111978F7309F4BFC00C9DC00190
:104CD0000D9D900D1124805E994FDC01AF54BE4FA5
:104CE00080559E4FFC018081879DF0011124EF5D6E
:104CF000F94F8381948123E0880F991F2A95E1F76A
:104D00002D913C91281739070CF49DC0C7010E94D2
:104D10008218C090CE08D090CF08C7010E947911A8
:104D20009601291B310937FF79C01092CF081092E4
:104D3000CE0835E0309320068FE08093CB0580E4E9
:104D40008093900082E893E290939900809398007A
:104D50008091CE089091CF08892B09F449C3E0E2F5
:104D6000F6E0FDA7ECA7FAA7E9A710E0112309F4E4
:104D7000DEC03FEF310F3EA78EA5A0E18A9FC001A4
:104D8000112499AB88AB29A43AA4712CD1019E9629
:104D90008C918E3009F073C27101BFE2EB0EF11CF1
:104DA0008090CA089090CB086090C808F10187A550
:104DB0000E945C0D29833A834B835C836D837E83E1
:104DC0008F83672D712FCE0101960E9465115C01C2
:104DD000C7010E942111582ED101D0968C918F3F8E
:104DE00009F04DC1EEECCE2EE7E0DE2E912C9614AC
:104DF00008F0D1C085E0F601DE01119601900D9218
:104E00008A95E1F78C819D8197FF93C09394B5E0DB
:104E1000CB0ED11CECCFF5E0FFA7E8CEC7010E9476
:104E20007911C91AD108D092CF08C092CE08CD28E6
:104E300009F47FCF45E04093CB05609290009092BB
:104E40009900809298001F5FEACE9C919F709630E7
:104E5000D1F70C9D90010D9D300D1124205E394F2E
:104E6000F901EF54FE4F20553E4FD9019C91979D7B
:104E7000D0011124AF5DB94F13962D913C91A3E061
:104E8000220F331FAA95E1F7408151814217530742
:104E9000D4F6F7012381348162819091DB089F73FE
:104EA000108291832A5031094091C8085091C90855
:104EB00042335105B0F4049FF001059FF00D112419
:104EC000E253F84F1082918362833483238380916D
:104ED000C8089091C90801969093C9088093C808A2
:104EE000B2CF70E04091C8085091C90884171506E8
:104EF00080F4809FF0011124E253F84F41814F73F9
:104F000031F41082918362833483238371E08F5F55
:104F1000E9CF711198CFD70111968C911197829595
:104F2000869586958370806411968C938CCF1EA68F
:104F300023CF8A818F7309F469CF69816F70C701AC
:104F40000E944A11882309F461CF61E276E0CE0124
:104F500001960E948711452DB5010E941112811101
:104F600055CFF10190AA87A5877C87A70E947C0F67
:104F7000D1019F968C919F978770823061F4D09673
:104F8000EC91E09FF0011124E253F84F808182956B
:104F90008F7009F03BCF8091CA089091CB08877041
:104FA0009927892B09F06BC164E0C7010E94F810B2
:104FB000882309F464C1812F173008F086E0442467
:104FC0004394480E55245A94570C711001C0512C2B
:104FD000872D3EE0371508F48EE099249394980EBF
:104FE000A8A8B9A86EA4852D90E099AF88AF81E0FC
:104FF000890DA82FB0E0BBAFAAAF461408F43FC19B
:1050000088AD99AD8A0D9B1D7C01EE0CFF1CE80E4E
:10501000F91EF701E05EF94F7F01852C2AAD3BAD0B
:105020002A0D3B1DC901880F991F820F931F9C01F8
:10503000225B394F3BAB2AAB3DAB2CABFC01E15BB8
:10504000F94FFFABEEAB981408F414C1781002C00E
:10505000161581F0D7019E968C918E3009F0D2C042
:105060006701BEE2CB0ED11CF70187A587708530A2
:1050700009F0E6C08394F3E0EF0EF11CE4CF809FCB
:10508000C0011124FC01E253F84F6F01DE011196BB
:10509000802F01900D928A95E1F78A818F7309F430
:1050A000ADC08C819D8197FDA9C0D1019F965C9078
:1050B000852D0E945C0D442E2AA33BA34CA35DA327
:1050C0006EA37FA388A761E0C7010E94F810882320
:1050D00009F459C082E0481A642D70E0C4010E94AE
:1050E0004A2C892B09F057CF852D90E063E09595E8
:1050F00087956A95E1F787708F5F38E0839FC001DD
:1051000011248873452D477C842BD1019F968C9365
:1051100090E073E0959587957A95E1F7B82FB77091
:105120005B2E09F038CF20E04CEC58E0B601C70107
:105130000E94F71EF10187A58770813031F1873019
:1051400021F1823011F42FEF20ABD101D0968C9158
:105150008F3F09F420CF61E276E0CE0101960E94F4
:1051600087116C01C7010E942111482FB501C601AA
:105170000E941112811142C08C819D8197FD3EC019
:105180000E947C0F08CF80E0A6CFD101D0968C91F1
:10519000809FC001112461E276E08253984F0E9403
:1051A00087114C015EECC52E57E0D52EF10180A988
:1051B000561458F68515E9F0D60111968C91119781
:1051C0008F73B9F013968D919C9197FD12C061E297
:1051D00076E0C6010E9487114CE0B4010E941112D2
:1051E000811107C021E04CEC58E0B601C7010E94D4
:1051F000F71E5394B5E0CB0ED11CD8CF2FEFF101A1
:1052000020ABC9CE981036CFFFE09F1609F432CFFD
:10521000CAA8DBA8ACA9BDA98C918E3009F02ACF11
:10522000EEA9FFA980810E945C0D29833A834B83FC
:105230005C836D837E838F832650223008F01ACFE3
:10524000D60111968C91282F30E093E03595279563
:105250009A95E1F72770263058F42E5F382F377C67
:10526000B8E02B9FC0011124832BF601818302CF6C
:1052700027E0F4CF639420E1A20EB11CBECE73945C
:1052800033E0230E311C40E1741280CD1F5F89A5ED
:105290009AA5C0969AA789A7183009F067CD2091E2
:1052A000C8083091C90880E08217130608F073C05F
:1052B000809FF0011124E253F84F91819F7309F010
:1052C00097C08F5FF1CFE530E1F480E28A8393E706
:1052D0009B839EE69C8394E69D839AE39E838F83C3
:1052E0008FE688878091D4089EE6811101C096E6FA
:1052F0009987882321F080E28A871B8621C186E670
:10530000FBCF82E089831CC18530E1F501E020E418
:1053100040E870E060E090E080E00E947A0C10923B
:10532000020181E08093A30104E110E01093A50144
:105330000093A4018AE090E09093A7018093A601D6
:105340008FEA97E00E94060C6091D00870E090E030
:1053500080E04AE00E94B118E0914D06F0E0EB5287
:10536000F74F9091D0088081891708F047C11093BA
:10537000A5010093A4011093A7010093A60183EA5D
:1053800097E03AC10E940C1939C11092AA017FC15D
:105390000E94410987C18091D0084091CC0850916A
:1053A000CD084B5F5F4F282F26952695240F352F6C
:1053B000311D3093CD082093CC088F5F8093D008A7
:1053C00082E0809320069FEFECA5FDA580E090ABE6
:1053D0008F5F33968031D9F71150ACA5BDA5D0961B
:1053E000BDA7ACA71111F0CF1092C9081092C80840
:1053F000BBA5BF5FBBA7EFA5EB13FACB0E94DC06F2
:105400001092A7011092A6011092A5011092A4017A
:1054100080912006811178CF01E020E440E870E01F
:1054200060E090E080E00E947A0C00E022E149E137
:1054300065E070E083E390E00E947A0CEE24E39450
:1054400002E129E145E558E065E070E083E390E0A2
:105450000E945A0902E020E043ED57E065E070E069
:1054600089E190E00E94930522E043ED57E065E07A
:1054700070E086E590E00E94930500E025E040E8BA
:105480006CE170E090E080E00E947A0CD12CC12C9D
:105490008FE0A82EB12C8091CA089091CB08B5015D
:1054A0000E944A2CEE24E39405E02FE044EC57E000
:1054B0006CE170E0D601A81BB90BCD010E945A091E
:1054C000BFE0CB0ED11CE6E9CE16D10421F7E09166
:1054D000D3081A821A8A1982E53008F0F4CE80E2E5
:1054E0008A838B839DE69C8391E69D8390E79E83D0
:1054F0008F8391E39E0F988789878A871B8692E620
:105500009A8B95E69B8B93E79C8B94E79D8B9AE314
:105510009E8B8F8BF0E0EB52F74F80811F928F9321
:1055200085E991E09F938F93CE0148969F938F9347
:105530000E94782C0F900F900F900F900F900F906B
:1055400000E02BE040E866E270E090E080E00E943E
:105550007A0C11E0109302011092A30186E190E011
:105560009093A5018093A40188E290E09093A70115
:105570008093A6016CE38CE196E00E94960B60E2BA
:105580008CE196E00E94960BCE0102960E94FF18D5
:1055900060E28CE196E00E94960B6EE38CE196E06F
:1055A0000E94960B109202011093A30182E090E0FA
:1055B0009093A5018093A40187E390E09093A701C5
:1055C0008093A601CE0142960E94FF1880914C065E
:1055D0008823A1F08091CA0882FD10C08FE290E07C
:1055E0009093A5018093A4018AE190E09093A70194
:1055F0008093A6018DEB97E00E94060C8091200617
:10560000843031F501E02CE24CE66AE070E08AE09B
:1056100090E00E947A0C2CE24CE66AE070E08AE0AE
:1056200090E00E944A0C1092020181E08093A30155
:1056300082E190E09093A5018093A4018CE190E039
:105640009093A7018093A60183E997E00E94060C3E
:1056500080912006853009F098CE6091D008809125
:105660004D0690E0FC01EB52F74F2081261778F4AD
:105670002091AA0121110BC085539F4F9A838983E2
:10568000CE0101960E94971F81E08093AA0180912C
:10569000D4089091A201891739F0882309F478CEB3
:1056A0000E9446090E947C0F0E945709B8C98F9238
:1056B0009F92AF92BF92CF92DF92EF92FF92CF93E1
:1056C000DF93EC01688179818A819B816115710585
:1056D0008105910521F464E279ED8BE597E02DE1F8
:1056E00033EF41E050E00E94DB2B49015A019B015E
:1056F000AC01A7EAB1E40E94FA2B6B017C01ACEE8D
:10570000B4EFA50194010E94082CDC01CB018C0DA3
:105710009D1DAE1DBF1DB7FF03C00197A109B04875
:1057200088839983AA83BB839F77DF91CF91FF9072
:10573000EF90DF90CF90BF90AF909F908F900895A3
:105740000E94572B08958FE091E00E94572B0895F7
:10575000B0E0A0E080930F0190931001A09311019D
:10576000B09312010895F999FECF92BD81BDF89AC8
:10577000992780B50895262FF999FECF92BD81BD56
:10578000F89A019700B4021639F01FBA20BD0FB67F
:10579000F894FA9AF99A0FBE0895262FF999FECF38
:1057A0001FBA92BD81BD20BD0FB6F894FA9AF99A3E
:1057B0000FBE01960895052E97FB1EF400940E94DB
:1057C000F22B57FD07D00E940D2C07FC03D04EF49E
:1057D0000C94F22B50954095309521953F4F4F4FAB
:1057E0005F4F089590958095709561957F4F8F4F8D
:1057F0009F4F08950E942F2CA59F900DB49F900D50
:10580000A49F800D911D11240895B7FF0C94FA2BCD
:105810000E94FA2B821B930B0895A1E21A2EAA1B59
:10582000BB1BFD010DC0AA1FBB1FEE1FFF1FA21750
:10583000B307E407F50720F0A21BB30BE40BF50B4D
:10584000661F771F881F991F1A9469F760957095D6
:10585000809590959B01AC01BD01CF010895A29F59
:10586000B001B39FC001A39F700D811D1124911D34
:10587000B29F700D811D1124911D0895991B79E02F
:1058800004C0991F961708F0961B881F7A95C9F7D0
:1058900080950895AA1BBB1B51E107C0AA1FBB1F1F
:1058A000A617B70710F0A61BB70B881F991F5A95AC
:1058B000A9F780959095BC01CD01089597FB072E1F
:1058C00016F4009407D077FD09D00E944A2C07FCFB
:1058D00005D03EF4909581959F4F08957095619500
:1058E0007F4F0895EE0FFF1F0590F491E02D09946E
:1058F000AEE0B0E0EEE7FCE20C94272F0D891E89A4
:1059000086E08C831A8309838FEF9FE79E838D83C4
:10591000AE01475E5F4F6F89788DCE0101960E9480
:105920009B2C2F813885020F131FF80110822E96B1
:10593000E4E00C94432FABE0B0E0E1EAFCE20C942D
:10594000192F7C013B018A01FC0117821682838199
:1059500081FFC8C1CE0101965C01F7019381F3017B
:1059600093FD859193FF81913F01882309F453C1F1
:10597000853239F493FD859193FF81913F01853202
:1059800029F4B70190E00E948B2EE7CF912C212CB7
:10599000312CFFE1F31538F08B3211F190F48032A5
:1059A00009F1833229F137FC3CC020ED280F2A3061
:1059B00050F536FE20C08AE0989E200D1124922ECC
:1059C00006C08D3291F0803371F7689430F8F3019E
:1059D00093FD859193FF81913F018111DACF21C021
:1059E000689431F8689432F8F2CF689433F8EFCFC6
:1059F000689434F8ECCFEAE02E9E200D1124222E7C
:105A0000689435F8E4CF8E3229F436FC04C16894EA
:105A100036F8DDCF8C3619F4689437F8D8CF88364D
:105A2000B1F2982F9F7D95549330E0F08336A1F129
:105A30008337C1F1833509F063C02801F2E04F0ECE
:105A4000511CF801C080D180692D70E036FC02C085
:105A50006FEF7FEFC6010E94752E4C01689437F8F6
:105A600082010AC00C5F1F4FFFE3F98388248394EF
:105A7000912C6501E89437F833FE2DC0522C811427
:105A8000910471F5552009F468CFB70180E290E0E8
:105A90000E948B2E5A94F6CFF801808189830E5F85
:105AA0001F4FE4CF2801F2E04F0E511CF801C080D7
:105AB000D180692D70E036FC02C06FEF7FEFC60128
:105AC0000E94802E4C018201D5CFB70180E290E088
:105AD0000E948B2E2A942814190409F0B0F7CECF17
:105AE000F60137FC859137FE81916F01B70190E097
:105AF0000E948B2E51105A94F1E08F1A9108BFCF5B
:105B0000843619F0893609F077C0F80137FE6BC08A
:105B100060817181828193810C5F1F4FF32DFF762D
:105B20003F2E97FF09C090958095709561957F4FA6
:105B30008F4F9F4F689437F82AE030E0A5010E940C
:105B4000BB2EC82ECA188C2C432C36FE0CC0E894F1
:105B500040F8C91440F434FE05C032FC03C0F32DF4
:105B6000FE7E4F2E892C44FE95C0FE01EC0DF11DEA
:105B70008081803309F087C0242D297E422E842D18
:105B80008870582E43FC95C040FE8FC09C2C821418
:105B900018F42C0C922C981844FE91C0B70180E3A5
:105BA00090E00E948B2E42FE09C088E790E041FE03
:105BB00002C088E590E0B7010E948B2EC91408F45A
:105BC0008AC0CA94D12C9FEFC91AD90ACA0CDB1C0F
:105BD000F60182916F01B70190E00E948B2EAC1408
:105BE000BD04B1F74FCF60817181072E000C880B87
:105BF000990B0E5F1F4F92CFD32CE894D4F82AE074
:105C000030E0853739F1232D297FD22E8F3601F1EF
:105C100048F48835A9F0F701868197812B96E2E157
:105C20000C94352F803749F08837A9F7D4FE02C08D
:105C30006894D2F820E130E00DC06894D4F8F6CF33
:105C400034FE03C0822F8660D82E20E132E002C0ED
:105C500028E030E0F801D7FE0FC0608171818281B9
:105C600093810C5F1F4FA5010E94BB2EC82ECA183E
:105C70003D2CE89437F867CF6081718190E080E037
:105C80000E5F1F4FF0CF42FC02C0839478CF839405
:105C9000839475CF842D867809F471CFF6CFB70140
:105CA00080E290E00E948B2E83948214C0F3512CEA
:105CB00073CF522C5818821408F46ECFF8CF842D6D
:105CC000867809F47BCF8BE241FE80E247FC8DE2CF
:105CD000B70190E071CFB70180E390E00E948B2E76
:105CE0009A946CCF8FEF9FEF99CFFC010590615094
:105CF00070400110D8F7809590958E0F9F1F0895E2
:105D0000FC016150704001900110D8F7809590958A
:105D10008E0F9F1F08950F931F93CF93DF93182F1C
:105D2000092FEB018B8181FD09C01FEF0FEF812F40
:105D3000902FDF91CF911F910F91089582FF14C092
:105D40002E813F818C819D81281739073CF4E881A1
:105D5000F981CF0101969983888310838E819F8179
:105D600001969F838E83E3CFE885F985812F09957E
:105D7000892BA1F3DACFFA01AA27283051F120317B
:105D800081F1E8946F936E7F6E5F7F4F8F4F9F4FCF
:105D9000AF4FB1E03ED0B4E03CD0670F781F891F11
:105DA0009A1FA11D680F791F8A1F911DA11D6A0FDF
:105DB000711D811D911DA11D20D009F468943F9192
:105DC0002AE0269F11243019305D3193DEF6CF0191
:105DD0000895462F4770405D4193B3E00FD0C9F757
:105DE000F6CF462F4F70405D4A3318F0495D31FDC4
:105DF0004052419302D0A9F7EACFB4E0A695979517
:105E0000879577956795BA95C9F7009761057105EC
:105E100008959B01AC010A2E069457954795379536
:105E20002795BA95C9F7620F731F841F951FA01D90
:105E300008952F923F924F925F926F927F928F922E
:105E40009F92AF92BF92CF92DF92EF92FF920F9309
:105E50001F93CF93DF93CDB7DEB7CA1BDB0B0FB613
:105E6000F894DEBF0FBECDBF09942A8839884888D0
:105E70005F846E847D848C849B84AA84B984C88466
:105E8000DF80EE80FD800C811B81AA81B981CE0F5D
:105E9000D11D0FB6F894DEBF0FBECDBFED01089542
:045EA000F894FFCFA4
:105EA400141001FFFFFFFF00E100000000000001EB
:105EB40000000000C18081000000080004060A0000
:105EC40007030B050C090D001E0602080201011B45
:105ED4000802080200021A07001101020323080441
:105EE4001E0003043C05032D0102051908023C00B1
:105EF4000406280407640201072606086402000059
:105F040000000047076E0868075D07AE076C078A44
:105F14000700000000890F00000000C30F0000000C
:105F240000F70F00000000A91000000000960B0904
:085F3400096C126B12256400D8
:00000001FF
